:020000040000FA
:020000000828CE
:08000800C62ECB2C8A018200F8
:10001000FF30A200FF30A300EA240A301926241181
:100020006D260330E124323032260330E1243230B1
:1000300032260330E124323032263230D5242830C3
:10004000D524812465247F2422128C26A317882698
:1000500023178926A3168A2623168B26A60103308A
:10006000A700A8010330A90007309F00BB24241675
:100070006B260130BD00BE01C201061F5C28861F31
:100080005C28BA01B9010130BD00C301C401C5013A
:100090005423BB240530B7246D30CD246530CD24E6
:1000A0006D30CD243D30CD246330CD246C30CD2453
:1000B0007230CD240130FD250230B7243630CD24F6
:1000C0003230CD243830CD245F30CD243530CD24AE
:1000D0003530CD243130CD243130CD242030CD24E5
:1000E0005630CD243030CD243130CD24013004269B
:1000F0000130B3246630CD247230CD246530CD2458
:100100006430CD246430CD246F30CD247330CD24C1
:100110007030CD246130CD246730CD246530CD24BE
:100120002E30CD246E30CD246C30CD240130FD2511
:100130000430B600B030B5006530B7009030B8007C
:100140003023762243222012BC01BB24C323061B8A
:10015000AD28861BAD28861AAE28B028A122A72874
:10016000061EB328C720061FB928861EB9283222CA
:10017000BA282322861FC028861EC0280E22C12826
:10018000FF21EF22201AC5287023A728C628BB24E8
:10019000061ACB28F3290030B7244D30CD24653022
:1001A000CD246E30CD247530CD24861E2F2900300D
:1001B000B3247330CD247430CD246530CD24703019
:1001C000CD243A30CD24861EE628BE0A04303E02F5
:1001D000031CEB28BE01BE08031DFB280130BD0037
:1001E000F7210630B3242E30CD243030CD243530E5
:1001F000CD242030CD243E08013C031D0C290230C3
:10020000BD00F7210630B3242E30CD243130CD246B
:100210003030CD242030CD243E08023C031D1D2962
:100220001430BD00F7210630B3243130CD242E30F8
:10023000CD243030CD242030CD243E08033C031D96
:100240002E29C830BD00F7210630B3243130CD242B
:100250003030CD242030CD242030CD245423013023
:100260001226061F92290130C5000030B3246930E0
:10027000CD246630CD242B30CD242030CD243A300F
:10028000CD24061F4429C20A04304202031C492916
:10029000C201C208031D5929C301C401F721063058
:1002A000B3243030CD243030CD242E30CD24303026
:1002B000CD244208013C031D6B29C301D630C40084
:1002C000F7210630B3243130CD243030CD242E3008
:1002D000CD243730CD244208023C031D7E29033053
:1002E000C3000A30C400F7210630B3243330CD24D4
:1002F0003830CD242E30CD243930CD244208033C73
:10030000031D91290730C300D030C400F721063007
:10031000B3243130CD243030CD243030CD242030C2
:10032000CD244322861FF129C5010030B324693052
:10033000CD246630CD242D30CD242030CD243A304C
:10034000CD24861FA429C20A04304202031CA92915
:10035000C201C208031DB929C301C401F721063037
:10036000B3243030CD243030CD242E30CD24303065
:10037000CD244208013C031DCB29C301D630C40063
:10038000F7210630B3243130CD243030CD242E3047
:10039000CD243730CD244208023C031DDE29033032
:1003A000C3000A30C400F7210630B3243330CD2413
:1003B0003830CD242E30CD243930CD244208033CB2
:1003C000031DF1290730C300D030C400F7210630E7
:1003D000B3243130CD243030CD243030CD24203002
:1003E000CD244322C82801300B26BB24C32B0A305E
:1003F000B3244D30CD244830CD247A30CD2C29087B
:10040000280203180C2A861F0C2AA80A2808290289
:10041000031D0B2A0E220D2AA8010800762220199E
:10042000222A3A08C6003908C700C8013D08C90099
:100430001D254A08BA004B08B900A011A01E212AA8
:10044000A01543220800270826020318302A061F99
:10045000302AA60A26082702031D2F2A3222312A13
:10046000A60108007622A018422A3A08C6003908D8
:10047000C700C8013D08C9008B254A08BA004B08CF
:10048000B900432208003608C6003508C7003A08FC
:10049000C8003908C9008B254A08AB004B08AA00E0
:1004A000542320124508013C031D642A2B08C60072
:1004B0002A08C7004308C8004408C9008B254A0819
:1004C000C1004B08C000752A2B08C6002A08C700C7
:1004D0004308C8004408C9001D254A08C1004B084C
:1004E000C000A011A01E752AA015BD2B37082B0235
:1004F000031C842A38082A02031C842AA014370803
:10050000AB003808AA00852AA0102B083602031C6D
:10051000932A2A083502031C932A20153608AB00BB
:100520003508AA00942A2011CA303D02031C9A2AD9
:100530000130BD000A304302031CA02AC401C301DC
:1005400008004008B3004108B4003308C60034086E
:10055000C7001430C800C901F6244608B300470894
:10056000B4004A08AE004B08AF002F08C9002E089F
:1005700089244608B0004708B1004808B20000309E
:10058000B3240430C6003108C70020309F25043052
:10059000C6003208C70030309F252E30CD240430ED
:1005A000C6003308CA000530CB00B7264C08C90086
:1005B0004908C7003030B3254D30CD244830CD2414
:1005C0007A30CD242D30CD243E30CD247030CD2452
:1005D0006C30CD246C30CD2401300426C32B2A0886
:1005E000B3002B08B4003308C6003408C700143029
:1005F000C800C901F6244608B3004708B4004A08F9
:10060000AC004B08AD002D08C9002C088924460811
:10061000B0004708B1004808B2000030B7240430E9
:10062000C6003108C70020309F250430C6003208BC
:10063000C70030309F252E30CD240430C60033084B
:10064000CA000530CB00B7264C08C9004908C700CE
:100650003030B3254D30CD244830CD247A30CD2CE8
:100660000130C60061264708B9000230C600612685
:100670004708BA000330C60061264708BF000430AF
:10068000C60061264708BD000530C6006126470840
:10069000C4000630C60061264708C3000730C60004
:1006A00061264708C50008000130C60039084B26FE
:1006B0000230C6003A084B260330C6003F084B26DE
:1006C0000430C6003D084B260530C60044084B26C2
:1006D0000630C60043084B260730C60045084B2E9F
:1006E0006130C70001244808C600461F8F2B0B301D
:1006F000B7244C30CD246F30CD246330CD246B3003
:10070000CD246130C700CE30C8000130F723241259
:100710006B260F30B7242A30CD242016952B2416B3
:100720006B260F30B7242030CD24BB0101301926B1
:10073000461B9D2BBB0A013019263B08323C03198E
:10074000A52B861BA52B061FBC2B0B30B7242030F6
:10075000CD242030CD242030CD242030CD24BC0128
:1007600024166B266130C700CE30C8000030F72356
:100770000F30B7242030CD2408006130C700410875
:10078000C8004008F72B0030B3242030CD2420309F
:10079000CD244630CD243630CD243230CD243830EF
:1007A000CD242030CD245030CD244C30CD244C30BD
:1007B000CD242030CD242030CD242030CD24203035
:1007C000CD2401304402031CEE2B0C30B3245230F4
:1007D000CD247830CD242030CD24F62B0C30B3241A
:1007E0005430CD247830CD242030CD240800C900E9
:1007F00047080824480822243324490822243324A3
:10080000652CC80047080E2415244908C8002F2C61
:10081000CA00722403104A0D2224332CC90072240A
:100820000310490D013E2224332CC9000830CA00B0
:100830000310C90D41244910A01E1F2C4914CA0BD6
:10084000182C0800CB000830CC00A012CB1F292C9C
:10085000A01654240310CB0DCC0B252C08003124FA
:10086000652CA012542C7F24221490267F24A214DD
:100870008F267F2485183D2C3A2C7F24A2108F26AA
:100880007F2C7F24221490267F24A2148F267F247D
:1008900085184B2C482C7F24A012051C502CA01628
:1008A0007F24A2108F267F2C7F242210A01E592C7B
:1008B000221490267F24A2148F267F248518612C71
:1008C0005E2C7F24A2108F267F2C7F24221090265E
:1008D0007F24A2108F267F24A2148F267F24221427
:1008E00090267F2C7F24221490267F24A2148F260A
:1008F0007F24221090267F24A2108F267F2C0C307C
:100900003E2EA4106E26A2108F2624106F262210D1
:10091000902ECA00C601C701C8011030CB0048089C
:10092000A3244C08C8004708A3244C08C700460865
:10093000A3244C08C600CA0DC90DC80DC70DC60DAD
:10094000CB0B8F2C0800CC004C08033ECD00CD1DF6
:10095000AB2C4D08CC004C08303ECD00CD1FB22C46
:100960004D08CC000800C6004608C03ED52CC70084
:100970004708803ED52C0830D5240130D524C83016
:1009800032260230D524C83032260630D5240C3029
:10099000D524C830322E2108CE00CE0024156D2675
:1009A0004E0E0F39E1244E08E12CC80024116D26AB
:1009B000480E0F39E124823032264808E124823083
:1009C000322ECF00A4156C264F087026A4116C2679
:1009D000FA303E2E0030702624116D26A4116C26AC
:1009E00000307F2622118E26A2118D2ECB00CA0147
:1009F000CB010130CC00CD01C91B042D0310CC0D5F
:100A0000CD0DC80DC90DFC2C48084602CE000030A3
:100A1000031C013049074702031C152DC7004E086F
:100A2000C6004C08CA074D08CB070310C90CC80CF8
:100A3000CD0CCC0C031C042D0800460848020318FA
:100A4000442DA0164708490203182D2D48084602D8
:100A5000CA0049084702CB00432D47084902031D3D
:100A6000362D48084602CA00CB01432D49084702EB
:100A70000318432D48084602CC0001304C02CA003E
:100A800049084702CB008A2D46084802031D642D01
:100A9000470849020318522DCA0149084702CB00F2
:100AA000A016632D47084902031D5A2DCA01CB0128
:100AB000A016632D490847020318632DCA01470891
:100AC0004902CB00A0128A2D4808460203188A2D3D
:100AD000A012470849020318772D46084802CC00A7
:100AE00001304C02CA0047084902CB008A2D470852
:100AF0004902031D802D46084802CA00CB018A2DF9
:100B00004908470203188A2D46084802CA004708C8
:100B10004902CB000800CB004708FF3CCC00490845
:100B20004C020318982D46084807013ECA009B2D29
:100B300046084807CA0047084907CB000800C80014
:100B40004608CB00470E0F39CC004808DE254D087B
:100B5000C8004608CB0047080F39CC004808DE25FE
:100B60004D08C8000800C8004708CB006430CC001E
:100B700097264D08C9004908C7004608CB0047081A
:100B8000CE000A30CF00A6265008CD004D08CC007C
:100B90004808DE254D08C8004708CB000A30CC00C5
:100BA00097264D08CA004A08C7004608CB004708E8
:100BB000CC004808DE254D08C8000800CD00CC0850
:100BC000031DEA2DCD080319E92D4D08A1004B0A9C
:100BD0000620FC2D0A304C020318F42D4C08303E40
:100BE000A1004B0A0620FA2D0A304C02413EA1001A
:100BF0004B0A06203030CD000800C6004608C80069
:100C00006430C9006430202EC6004608C800643035
:100C1000C9003230202EC6004608C8006430C90022
:100C20001430202EC6004608C8006430C9000A30BF
:100C3000202EC7004708C8006430C9000130202EAC
:100C4000CA00FF30CB004908CD004808CC0017305F
:100C50004B070318282ECC0B272ECD0B252ECA0BA5
:100C6000232E0800C9004908CA00CA08031D392EEE
:100C70003D2E0A303E26CA03352E0800D000F4303F
:100C8000D100FC30D20050085107031C0034520739
:100C90000318472E0800C7004608831603139B005D
:100CA0008312470883169A001C158B1355309D003C
:100CB000AA309D009C149C185B2E1C118B1783126C
:100CC0000800C7004608831603139B001C141A086B
:100CD0008312C70008007C2E7C2E7C2E7C2E7C2E5E
:100CE000D00050080F39D1002508F0395104A50073
:100CF000792E250886000800240885000800A60033
:100D000026080F39A7002308F0392704A300912EE5
:100D1000912E912E912E912E942E942E942E942ECF
:100D2000942E230866000800220865000800CC08FD
:100D30000319A32E4C084B0203189F2EA32E4C0818
:100D40004B02CB009A2E4B08CD000800D101CF08F2
:100D50000319B42E4F084E020318AF2EB42E4F08BD
:100D60004E02CE00D10AAA2E5108D0000800CD01B3
:100D70004B08003C031CBD2EC32E4A08CD07013092
:100D80004B02CB00B82E4D08CC0008000430A10067
:020D9000080059
:02400E00613F10
:00000001FF
